:103D78000FC30FBF0FBB0FB60FB20FAC0FA70FA12A
:103D88000F9B0F950F8E0F870F800F780F700F689E
:103D98000F5F0F550F4B0F410F360F2B0F1F0F12D1
:103DA8000F060EF80EEA0EDB0ECC0EBC0EAB0E9A0A
:103DB8000E880E750E620E4E0E390E240E0E0DF77D
:103DC8000DDF0DC70DAE0D940D790D5E0D410D245F
:103DD8000D070CE80CC90CA90C890C680C460C23BF
:103DE8000C000BDC0BB80B930B6E0B480B210AFA7B
:103DF8000AD30AAC0A840A5B0A330A0A09E109B73A
:103E0800098E0965093B091108E808BE0895086C80
:103E18000842081907F107C807A0077807500729BB
:103E2800070206DB06B5068F066A0645062105FD6C
:103E380005DA05B70595057405530532051204F32F
:103E480004D404B60498047B045F04430428040DD6
:103E580003F303DA03C103A90391037A0363034D50
:103E680003370322030E02F902E602D302C002AEB0
:103E7800029C028B027A026A025A024B023C022D11
:103E8800021F0211020301F601E901DD01D001C59B
:103E980001B901AE01A30198018E0184017A017173
:103EA8000168015F0156014D0145013D0135012EB3
:103EB8000126011F01180111010B010400FE00F881
:103EC80000F200EC00E600E100DC00D600D100CCF6
:103ED80000C800C300BE00BA00B600010C0101040E
:103EE80002011E030A960401320503030600640753
:103EF800010108000009015A0E01010F000112001A
:103F08006413010114013C1501FA1664FA17FFFF46
:103F18001D00072000072400022701012F013C3063
:103F2800010132010335FFFF3603073CFFFF3DFF68
:103F3800FF180002191E461A00021B00022D32C883
:103F48002E0001FAFAFA18000019FFFF1A00001BE8
:103F580000002D32C82E0001FAFAFA18000019FFE5
:103F6800FF1A00001B00002DFFFF2EFFFFFAFAFAD0
:10004800900786E0FEA3E0FF7457BE0010D39F40E0
:100058000C903EE212001EE493F599804C90001437
:10006800E0D394044014900786E0FEA3E0FF903E9E
:10007800E212001EE493F599802F900014E0D394C7
:10008800034014900786E0FEA3E0FF903EF71200BD
:100098001EE493F5998012900786E0FEA3E0FF9096
:1000A8003F0C12001EE493F59990078612000E90FB
:1000B8000786E0FEA3E0FF746C6F4E7003751300B3
:1000C80022900072E0B402087401900072F0D20C21
:1000D80090013AE090002AF090013BE090002BF06C
:1000E80090013CE090002CF0A20AB3401690013A2F
:1000F800E0700C90013BE0700690013CE0600280EB
:1001080002C20A90013AE0B4300F90013BE0B447D4
:100118000890013CE0643B60028004D20B8002C27C
:100128000BE557B40102800302024B900057E0F53B
:1001380065900062E0F567900063E0F568900074F0
:10014800E0F56990007AE0900029F090007CE0F5F5
:100158006490007DE0F566900080E0F56390008192
:10016800E0F562900090E0900041F0900091E090FE
:100178000042F0900092E0900043F0900093E090ED
:100188000044F0900094E0900045F0900095E090D5
:100198000046F0900096E0900047F0900097E090BD
:1001A8000048F0900099E0900033F090009AE090B9
:1001B8000034F090009BE0900035F090009CE090B7
:1001C8000036F0900079E0B4011790000A740FF03F
:1001D800A374FFF090000CE4F0A3F074029000798F
:1001E800F0900079E0B4035990000CE0FEA3E0FF22
:1001F80090000AE0FCA3E0FD12000374101240D83E
:1002080074081240CAEF900026F0EF700674FF9051
:100218000026F07400900079F090000BE090002721
:10022800F090000AE0900028F0900026E0900789FE
:10023800F0900027E090078AF0900028E090078B64
:10024800F0803F900081E07006755701756200A24A
:100258000AB3402E90013AE090002AF090013BE06A
:1002680090002BF090013CE090002CF090002AE0E8
:10027800700C90002BE0700690002CE06002800269
:10028800C20AE5657003756502E567700375670264
:100298007E837FC2E5658E048F05FF1240BA8C38D5
:1002A8008D39E56875F0FAA4FFAEF0E5678E048F26
:1002B80005FF1240BA8C3C8D3D90004FE0F55F90F1
:1002C800004DE0FE900069E0B5061890004CE0FE95
:1002D800900068E0B5060C90004BE0FE900059E0F5
:1002E8006E606F900069E07006900068E0600674C8
:1002F80000900059F0900069E0B402089000497439
:1003080001F08005900049E4F0900068E0B402082C
:1003180090004A7401F0800590004AE4F09000686B
:10032800E0600690004AE060028005755F03800384
:10033800755F04E558B55702D20C900068E090004C
:100348004CF0900069E090004DF0900059E090006A
:100358004BF0740190009EF0740190009FF07400BF
:100368009000A0F074009000A1F074009000A2F03A
:1003780074009000A3F074009000A4F07401900041
:10038800A5F074019000A6F074009000A7F0740026
:100398009000A8F074009000A9F074009000AAF0F2
:1003A80074009000ABF074019000ACF07401900000
:1003B800ADF074009000AEF074009000AFF07400DF
:1003C8009000B0F074009000B1F074009000B2F0AA
:1003D8007401900362F07401900363F07400900359
:1003E80064F07400900365F07400900366F0740084
:1003F800900367F07400900368F074009003A2F013
:1004080074019003A3F074009003A4F074009003A7
:10041800A5F074009003A6F074009003A7F0740090
:100428009003A8F074009003E2F074009003E3F0E6
:1004380074009003E4F074009003E5F074009003F6
:10044800E6F074009003E7F074009003E8F074019C
:10045800900422F07400900423F07400900424F0B7
:100468007400900425F07400900426F07400900441
:1004780027F07400900428F022E5B554F7F5B5E5A7
:10048800B554FDF5B5C2A2C2A1C292C207E5B554E2
:10049800FBF5B5755004E55004F55190004FE0F5B3
:1004A8005F900025E4F0C209E5B554FEF5B5227564
:1004B8000A00750900AE09AF0A7457BE00039F50C1
:1004C80003020574903EE212001EE49390004E125F
:1004D80040F00FBF00010EE0FC903EE212001EEC5F
:1004E800FEE493FFEEC39F5026AE09AF0A0FBF008C
:1004F800010E903EE212001EAE09AF0AE493FC9092
:100508003EE212001EE49390004E1240F0ECF0AE72
:1005180009AF0A903EE212001EE49390004E12408A
:10052800F0E0FC903EE412001EECFCE493FDECD3FA
:100538009D4019903EE412001EE493FC903EE212A6
:10054800001EE49390004E1240F0ECF0AE09AF0AA2
:1005580074022FFF50010E8E098F0A780A74012643
:10056800F6500418E436F640030204BD22750A006A
:10057800750900AE09AF0A7415BE00039F50030247
:100588000642903F3912001EE49390004E1240F04C
:100598000FBF00010EE0FC903F3912001EECFEE494
:1005A80093FFEEC39F5026AE09AF0A0FBF00010E9E
:1005B800903F3912001EAE09AF0AE493FC903F3910
:1005C80012001EE49390004E1240F0ECF0AE09AF1A
:1005D8000A903F3912001EE49390004E1240F0E05A
:1005E800FC903F3B12001EECFCE493FDECD39D40D5
:1005F80019903F3B12001EE493FC903F3912001EF5
:10060800E49390004E1240F0ECF0AE09AF0A740F7C
:100618006F4E7006750A15750900AE09AF0A7402A7
:100628002FFF50010E8E098F0A780A740126F650A2
:100638000418E436F6400302057B22750A007509A2
:1006480000AE09AF0A7415BE00039F5003020710DD
:10065800903F4E12001EE49390004E1240F00FBFE0
:1006680000010EE0FC903F4E12001EECFEE493FFEA
:10067800EEC39F5026AE09AF0A0FBF00010E903F90
:100688004E12001EAE09AF0AE493FC903F4E1200D2
:100698001EE49390004E1240F0ECF0AE09AF0A90C1
:1006A8003F4E12001EE49390004E1240F0E0FC9082
:1006B8003F5012001EECFCE493FDECD39D401990D2
:1006C8003F5012001EE493FC903F4E12001EE4932C
:1006D80090004E1240F0ECF0AE09AF0A740F6F4E66
:1006E8007006750A15750900AE09AF0A74022FFF66
:1006F80050010E8E098F0A780A740126F6500418E4
:10070800E436F6400302064922750A00750900AE70
:1007180009AF0A7415BE00039F50030207DE903F1D
:100728006312001EE49390004E1240F00FBF0001C8
:100738000EE0FC903F6312001EECFEE493FFEEC354
:100748009F5026AE09AF0A0FBF00010E903F6312FB
:10075800001EAE09AF0AE493FC903F6312001EE44A
:100768009390004E1240F0ECF0AE09AF0A903F6350
:1007780012001EE49390004E1240F0E0FC903F659A
:1007880012001EECFCE493FDECD39D4019903F65EC
:1007980012001EE493FC903F6312001EE493900045
:1007A8004E1240F0ECF0AE09AF0A740F6F4E7006AF
:1007B800750A15750900AE09AF0A74022FFF5001BA
:1007C8000E8E098F0A780A740126F6500418E4364A
:1007D800F6400302071722054C22054B22054DC29D
:1007E800CF2290F800E4936406600280FE758401CD
:1007F80075A70075FF80900788E4F075C91075A784
:100808000F75A1C775A70075D90075CEFF75A70F1D
:1008180075F1FE75F2FF75F33775F47875A4BA753E
:10082800A5FF75A60775AE0075AFFF75D48175D5A0
:10083800FF75D6FF75D7FFC296C295C2A0C297E5CD
:10084800B554BFF5B5E5B554DFF5B5E5B554EFF5E5
:10085800B5E5B5547FF5B5E5B554F7F5B5E5B55447
:10086800FDF5B575A70075A20175A14775F809755D
:10087800BC0175BE0475BD6C75BE0775BDA075BE9F
:100888000875BD0175BC0075BB1875BC2075BA0824
:1008980075E88075D11375A70F75E10575E20075C8
:1008A800C740759700759780740A1240AA7597C05B
:1008B800E5975420700280F8758F0275A700D2AFB3
:1008C80075980075A90C75A70F75AB4375ADFB75C9
:1008D800AC1E75A700758911758E00758C00758A18
:1008E80000D2A9D28C758D00758B00D2ABD28E75D3
:1008F800CD0075CC0075CA0075CB00D2ADC2CFD281
:10090800CA7591047592007593CD75EF0675D94037
:1009180075CF01900786E4F0A3F0751300751400F5
:10092800C299D20A74C8F5187517001226A175A7BE
:100938000FE5FB90001AF0E5FA90001BF0E5F9903E
:10094800001CF075A70090F800E493F5081227D86A
:10095800122D12900789E0900026F090078AE09007
:100968000027F090078BE0900028F090078CE0902B
:100978000029F090078DE0F56590078EE0F5679007
:10098800078FE0F568900790E0F569900791E0F52A
:1009980064900792E0F566900793E0F563900794FA
:1009A800E0F562900795E090002AF0900796E090B5
:1009B800002BF0900797E090002CF0900798E090BB
:1009C8000041F0900799E0900042F090079AE0907B
:1009D8000043F090079BE0900044F090079CE09063
:1009E8000045F090079DE0900046F090079EE0904B
:1009F8000047F090079FE0900048F09007A0E09033
:100A08000033F09007A1E0900034F09007A2E09046
:100A18000035F09007A3E0900036F0740090008253
:100A2800F090013AE0700C90013BE0700690013CB8
:100A3800E060028004C20A8002D20A90F807E493B8
:100A4800900021F0900021E0440A900021F09000ED
:100A580021E054FE900021F07406900012F0740218
:100A6800900013F090F802E493900014F07403904F
:100A78000015F07403900016F07412900017F074CB
:100A880005900018F0900014E0B404067404900077
:100A980018F0900014E0B403067403900018F07482
:100AA80004900019F090F804E49390001DF074008D
:100AB80090001EF090F805E49390001FF090F8065F
:100AC800E493900020F074FF900022F0744A9001A3
:100AD80025F07461900126F07474900127F0746316
:100AE800900128F0746F900129F0742090012AF089
:100AF800745290012BF0744590012CF074349001DD
:100B08002DF0742090012EF0742090012FF0743491
:100B1800900130F07453900131F07450900132F02C
:100B28007444900133F090007AE0D3940140067445
:100B38000090007AF0755701755801740390004CC5
:100B4800F01200C91204B7900014E0B404051206AC
:100B5800438011900014E0D3940440051205758079
:100B6800031207111226CDE5B554FEF5B590002500
:100B7800E4F0900786E4F0A3F07523007522007571
:100B880047007529007528007548007531007530D3
:100B98000075490075530075540075590075500467
:100BA80075510175333C753200756F00756E0075AF
:100BB80070CD755500755600754200754300754433
:100BC80000754500755A007546007541007540006E
:100BD800900006E4F0A3F0900008E4F0A3F0755D3F
:100BE80000755E0090000E74FDF0A374E8F09000AC
:100BF80023E4F07464900024F0C200D201C202D24F
:100C080003754C00756C00C294C293C287C290C22F
:100C180091C20C7E017F00900028E01240D890001D
:100C280027E02FFF50010E90000AEEF0A3EFF0909E
:100C38000026E0700674FF900026F090000AE0FE9F
:100C4800A3E0FFEFD394FFEE940F400790000AE46F
:100C5800F0A3F07400900071F07400900079F074C3
:100C680000900082F0740090008DF074009000B441
:100C7800F0E5667003756604743A90074EF074FDEB
:100C880090074FF09003D4E0900414F0D2B0D2B79C
:100C9800D2A7D2A6D2B1D2A3C207A2B6B39204A257
:100CA800B3B39205D29CD2EC75CF01A298B340059C
:100CB800C298123076E5136006A299B3B340028059
:100CC80005C2991235ECE51464016005E514B40415
:100CD8000280D5E54CD39405400CE559C394C8501F
:100CE800020559754C00E570C394F0501A786E12DD
:100CF800003FAE6EAF6FEFD394E8EE940340080563
:100D080070756F00756E00C28E7E047F00E54B1211
:100D180040D8E58D75F004A4FDACF0EF2DFDEE3C58
:100D2800FCE58B75F04084FF7E00ED2FFFEC3EFE66
:100D38008E248F25D28EA2B6300401B35003020E42
:100D480076A2B6300401B35003020E76A2B6405A1A
:100D58000553E5B54401F5B5900024E4F0E553D317
:100D6800956540447C837DC2123F788E228F23E5AF
:100D7800472FFF50010E74011240CA8E228F23851F
:100D88002347755301C28E758D00758B00754B0016
:100D9800D28E7403BE00039F50069000257401F0A4
:100DA800E542B40603754200D204A2B6B35003026A
:100DB8000E76C20490006BE0601812372DA200B3C3
:100DC8004008E5B54408F5B58006E5B554F7F5B52E
:100DD8008002C20090006EE06018123882A202B34E
:100DE8004008E5B54402F5B58006E5B554FDF5B50E
:100DF8008006E5B554FDF5B5A207B34004D2878057
:100E080002C287900059E06004D2908002C290909C
:100E1800004AE0B40104D2948002C294900049E0F0
:100E2800B40104D2938002C293A209B34004D291C0
:100E38008002C291900018E0FE900014E0C39E402A
:100E480009900014E0D39408400974FB900023F043
:100E580012048190001DE0601590001DE0FE9000D6
:100E680017E06E600974FE900023F0120481C2CA74
:100E78007E017F00E54D1240D8E5CD2FFF50010ED1
:100E88008E268F27D2CAE564B4014890000EE0FC94
:100E9800A3E0FDEFC39DEE9C4039B208E529452843
:100EA8006013A208B34008E5B54404F5B58006E52B
:100EB800B554FBF5B590000EE0FEA3E0FF900010DE
:100EC800E0FCA3E0FDEF2DFDEE3CFC90000EECF005
:100ED800A3EDF0A2B3300501B35003020FBBA2B3D8
:100EE800300501B35003020FBBA2B35003020FB485
:100EF8000554E5B54401F5B5900024E4F0E554D374
:100F080095675003020FB27CEA7D60AE26AF2712C8
:100F18003F788E288F29E5681240D874FF8E048F99
:100F280005FF1240BA8C288D29E5482DFD50010C8B
:100F380074018C068D071240CA8E288F298529488E
:100F4800A209B3401574641240D8900067E08E047B
:100F58008F05FF1240BA8C288D2975540190000E18
:100F6800E0FEA3E0FFAC26AD2712000390000EEED2
:100F7800F0A3EFF0E566FF1240BA740AFF1240BA18
:100F880090007BE08C068D071240D874148E048F75
:100F980005FF1240BA900010ECF0A3EDF0C2CA753C
:100FA800CD0075CC00754D00D2CAD205A2B3B340AE
:100FB80002C205900025E0B40107E555C394064038
:100FC800030215CFE56C902665F828287390005920
:100FD800E0C394024003021129E550D39401500361
:100FE800021129E55075F040A4FFAEF090031212EB
:100FF800001EE0C395445018E55075F040A4FFAEBC
:10100800F090031112001EE0F52D752C0002112935
:10101800E55075F040A4FFAEF090031012001EE0FA
:10102800C3954440030210C5E55075F040A4FFAED7
:10103800F090031112001EE55075F040A4FFAEF0C9
:10104800E0FC90030F12001EECFEE0FFEEC39FFED3
:10105800E5508E0475F040A4FFAEF0900310120026
:101068001EE0F40425448C0088F0A4FFAEF0E5509F
:101078008F048E0575F040A4FFAEF09003121200A5
:101088001EE55075F040A4FFAEF0E0FA9003101290
:10109800001EEAFEE0FFEEC39FFECDCCCD8E071208
:1010A80040BAE55075F040A4FFAEF090030F12006F
:1010B8001EE02DFD50010C8C2C8D2D8064E55075A3
:1010C800F040A4FFAEF090030F12001EE55075F03B
:1010D80040A4FFAEF0E0FC90030E12001EECFEE010
:1010E800FFEEC39F8544F0A4FFAEF0E5508F048E59
:1010F8000575F040A4FFAEF090031012001EE0FE4C
:10110800CDCCCD8E071240BAE55075F040A4FFAEA5
:10111800F090030E12001EE02DFD50010C8C2C8D5A
:101128002D756C010215CF900059E0C3940240035D
:101138000212DD90004FE0D395505003021285E56E
:101148005075F040A4FFAEF090031812001EE0C3E3
:1011580095445018E55075F040A4FFAEF090031781
:1011680012001EE0F52B752A00021285E55075F075
:1011780040A4FFAEF090031612001EE0C395444051
:1011880003021221E55075F040A4FFAEF09003175A
:1011980012001EE55075F040A4FFAEF0E0FC90038D
:1011A8001512001EECFEE0FFEEC39FFEE5508E0414
:1011B80075F040A4FFAEF090031612001EE0F40490
:1011C80025448C0088F0A4FFAEF0E5508F048E050E
:1011D80075F040A4FFAEF090031812001EE550759C
:1011E800F040A4FFAEF0E0FA90031612001EEAFEEB
:1011F800E0FFEEC39FFECDCCCD8E071240BAE5507E
:1012080075F040A4FFAEF090031512001EE02DFD0E
:1012180050010C8C2A8D2B8064E55075F040A4FF9A
:10122800AEF090031512001EE55075F040A4FFAE15
:10123800F0E0FC90031412001EECFEE0FFEEC39FEA
:101248008544F0A4FFAEF0E5508F048E0575F0409C
:10125800A4FFAEF090031612001EE0FECDCCCD8E9A
:10126800071240BAE55075F040A4FFAEF0900314A1
:1012780012001EE02DFD50010C8C2A8D2BE550B478
:101288000123E55FD39401401CE55504D3955040F4
:1012980014E544C39405500D90035FE0A828B800F6
:1012A80006952940028003755002E550B55F2290EB
:1012B800004FE0D395504019E55075F040A4FFAEBB
:1012C800F090031712001EE0A822B80006952340EC
:1012D800028002055F756C020215CF900059E0B4D8
:1012E800022AE55075F040A4FFAEF09003171200F3
:1012F8001EE0F52B752A00E55075F040A4FFAEF00E
:1013080090030E12001EE0F52D752C00900059E098
:10131800B4030F900051E0F52B752A00752D007568
:101328002C00756C030215CFE55075F040A4FFAE94
:10133800F090032012001EE0C395594003021405E3
:10134800900049E07036E550D394014029AE22AFB1
:1013580023AC2CAD2DEDD39FEC9E401AE55075F0D3
:1013680040A4FFAEF090031E12001EE0A828B800AB
:1013780005D395295002800215508034E550D39446
:10138800024029AE22AF23AC2CAD2DEDD39FEC9EAD
:10139800401AE55075F040A4FFAEF090031E12000D
:1013A8001EE0A828B80005D39529500280021550E0
:1013B800E550B55137E550C3955F5030E55504D336
:1013C80095504028AE22AF23AC2AAD2BEFD39DEE2B
:1013D8009C4019E55075F040A4FFAEF090031F1231
:1013E800001EE0A828B80006952940028002055092
:1013F800C292E55065516005C207755900756C04C5
:101408000215CFE55075F040A4FFAEF090031A1214
:10141800001EE0B40117E55075F040A4FFAEF0904F
:10142800032012001EE0240AC3955940030214DB6E
:10143800752F64752E00A207B3500B900060E0244E
:1014480005C3954440030214DBE55075F040A4FF42
:10145800AEF090031D12001EE0C395444064E550B1
:1014680075F040A4FFAEF090031C12001EE5507505
:10147800F040A4FFAEF0E0FC90031B12001EECFE4F
:10148800E0FFEEC39F8544F0A4FFAEF0E5508F0463
:101498008E0575F040A4FFAEF090031D12001EE00B
:1014A800FECDCCCD8E071240BAE55075F040A4FFB2
:1014B800AEF090031B12001EE02DFD50010C8C2E87
:1014C8008D2FAE22AF23AC2EAD2FEFD39DEE9C40D7
:1014D80002D207756C050215CFE550B401099000DA
:1014E80059E0C3940240030215AF900358E0D39526
:1014F8004450030215AF900356E0C3954450409002
:101508000357E0FE900355E0F4042EFE900356E0E6
:10151800F40425448E0088F0A4FFAEF0900358E050
:10152800FC900356E0F4042C8E048F05FF1240BA99
:10153800900355E02DFD50010C8C2A8D2B802C90AA
:101548000355E0FE900354E0F4042E8544F0A4FF14
:10155800AEF0900356E08E048F05FF1240BA900358
:1015680054E02DFD50010C8C2A8D2BE550C3955F5E
:101578005030E55504D395504028AE22AF23AC2A0D
:10158800AD2BEFD39DEE9C4019E55075F040A4FFBC
:10159800AEF090031F12001EE0A828B80006952997
:1015A80040028003755002900049E0B40106E550FE
:1015B800640160028003755002E55065516005C200
:0715C80007755900756C0066
:10266500020FD502112F0212E302133002140B02DE
:0226750014E16E
:1015CF00900050E02402A822B80007D395234002D0
:1015DF00C207900025E0B40109900059E0C39403BD
:1015EF004003021757900049E060030216A6E5502A
:1015FF00D394014034E55075F040A4FFAEF0900352
:10160F001412001EE0A822B8001FD39523401AE53C
:10161F005075F040A4FFAEF090031F12001EE0A81B
:10162F0028B80005D39529500280021550E550D3F4
:10163F009401402FE55075F040A4FFAEF0900312D7
:10164F0012001EE0C39544501AE55075F040A4FFF8
:10165F00AEF090031E12001EE0A828B80005D39527
:10166F0029500280021550E550D394014022E555D0
:10167F0004C39550501AE55075F040A4FFAEF0909A
:10168F00031E12001EE0A828B80005D395295002AA
:10169F008002155002174CE550D394024034E550A8
:1016AF0075F040A4FFAEF090031412001EE0A822C4
:1016BF00B8001FD39523401AE55075F040A4FFAE34
:1016CF00F090031F12001EE0A828B80005D395293B
:1016DF00500280021550E550D39402402FE550750B
:1016EF00F040A4FFAEF090031212001EE0C3954429
:1016FF00501AE55075F040A4FFAEF090031E120093
:10170F001EE0A828B80005D3952950028002155075
:10171F00E550D394024022E55504C39550501AE585
:10172F005075F040A4FFAEF090031E12001EE0A80B
:10173F0028B80005D39529500280021550E5506551
:10174F00516005C207755900900060E0D395445071
:10175F0009900054E0C395445002C207900059E02D
:10176F0070030219BCA2A5B34008A2A4B3400302A0
:10177F0019A5AE34AF357441D39F749C9E40057844
:10178F003412003FAE34AF35EFB48806EEB4130217
:10179F008003021982A2A55003021845900059E058
:1017AF00B4010B90004FE0D3955F4002055F9000AE
:1017BF0059E0B40254E55075F040A4FFAEF0900329
:1017CF002012001EE0C39559503F90004FE0D39573
:1017DF00504021E55504D395504019E55075F04020
:1017EF00A4FFAEF090031412001EE0A822B800066A
:1017FF00952340028002055090004FE0F55FE550C1
:10180F0065516005C207755900900059E0B4032671
:10181F0090004FE0D395504008E55504D3955050B4
:10182F00028002055090004FE0F55FE55065516072
:10183F0005C207755900A2A45003021982900059DE
:10184F00E0B4016E900049E07035E550D39401404B
:10185F0029E55075F040A4FFAEF090031E12001E54
:10186F00E0A828B8000FD39529400A1550755900E4
:10187F0085505F800385505F8003755F018033E57E
:10188F0050D394024029E55075F040A4FFAEF0907C
:10189F00031E12001EE0A828B8000FD39529400A96
:1018AF00155075590085505F800385505F80037513
:1018BF005F02900059E0D394015003021976E5506E
:1018CF0075F040A4FFAEF090032012001EE0C39508
:1018DF00594003021976900049E07041E550D394C6
:1018EF00014034E55075F040A4FFAEF090031112A3
:1018FF00001EE0A822B8001FD39523401AE55075AB
:10190F00F040A4FFAEF090031E12001EE0A828B80E
:10191F000005D39529500280021550803FE550D322
:10192F0094024034E55075F040A4FFAEF0900311DF
:10193F0012001EE0A822B8001FD39523401AE550CD
:10194F0075F040A4FFAEF090031E12001EE0A82811
:10195F00B80005D39529500280021550E550655106
:10196F006005C207755900E555B40704055D80038E
:10197F00755D00E562B4010EAE34AF35EF644070B3
:10198F0005EE649C6002800EA2A54003755701A26C
:10199F00A44003755702A2A5B3B35006A2A4B3B3D4
:1019AF0040028006753500753400021AAAA2A5B34D
:1019BF004008A2A4B34003021A96AE34AF35744167
:1019CF00D39F749C9E4005783412003FAE34AF35E0
:1019DF00EFB48806EEB413028003021A96A2A54054
:1019EF006F900068E0605A90004AE0B401079000E1
:1019FF004AE4F0800690004A7401F090004AE070CB
:101A0F0005755F038003755F0490004AE0B401041D
:101A1F00D2948002C294E550B4041AE55075F04098
:101A2F00A4FFAEF090031E12001EE0A828B8000518
:101A3F00D3952950028008755003C207755900804D
:101A4F0003755F04E555B40704055D8003755D00FC
:101A5F00A2A44033900069E06021900049E0B401F6
:101A6F0007900049E4F080069000497401F090005F
:101A7F0049E0B40104D2938002C293E555B4070440
:101A8F00055D8003755D00A2A5B3B35006A2A4B394
:101A9F00B340028006753500753400E55765586010
:101AAF0006900082E06003021C32C29C7514007520
:101ABF001300C2CAE557902677F8282873801212B0
:101ACF002D12800D122DEB8008122EC48003122FC1
:011ADF009D69
:0F267700021ACC021ACE021AD3021AD8021ADDA6
:101AE000900029E090007AF0E565900057F0E567F6
:101AF000900062F0E568900063F0E569900074F092
:101B0000E56490007CF0E56690007DF0E563900070
:101B100080F0E562900081F090002AE090013AF0B8
:101B200090002BE090013BF090002CE090013CF005
:101B3000900041E0900090F0900042E0900091F021
:101B4000900043E0900092F0900044E0900093F009
:101B5000900045E0900094F0900046E0900095F0F1
:101B6000900047E0900096F0900048E0900097F0D9
:101B7000900033E0900099F0900034E090009AF0EB
:101B8000900035E090009BF0900036E090009CF0D3
:101B90007400900082F0744A900125F07461900105
:101BA00026F07474900127F07463900128F0746F2C
:101BB000900129F0742090012AF0745290012BF0CA
:101BC000744590012CF0743490012DF07420900134
:101BD0002EF0742090012FF07434900130F0745383
:101BE000900131F07450900132F07444900133F060
:101BF0009003D4E0900414F0743A90074EF074FD12
:101C000090074FF01200C9900004E4F0A3F0900098
:101C1000067475F0A37430F09000087475F0A37426
:101C200030F0855758D2CA754B00D29C741B900077
:101C300023F0E555C394065005E550B55102804E9A
:101C4000C207E55075F040A4FFAEF09003221200E9
:101C50001EE030E003D38001C39296E55075F0405A
:101C6000A4FFAEF090032312001EE030E003D38007
:101C700001C39295855051AE28AF297405BE00036B
:101C80009F5007E544D3940550028002D292E55557
:101C9000D394055003021D57C207E550D394014069
:101CA00059E55075F040A4FFAEF090031E12001EDF
:101CB000E0A828B80007D3952940021550E55065E3
:101CC000516035E55075F040A4FFAEF0900322124C
:101CD000001EE030E003D38001C39296E55075F01A
:101CE00040A4FFAEF090032312001EE030E003D3C7
:101CF0008001C39295855051805DE555B4061A90D8
:101D000000ACE030E003D38001C392969000ADE0D8
:101D100030E003D38001C39295E555B4071A9000D3
:101D2000A5E030E003D38001C392969000A6E03096
:101D3000E003D38001C39295E555B4081A90009E44
:101D4000E030E003D38001C3929690009FE030E042
:101D500003D38001C39295900072E06058E544750A
:101D6000F00284FF7E0090014E12001EE0F55BE55C
:101D70004675F00A84FF7E0090024E12001EE0F5C8
:101D80005CE55B255CD39464400BE55B255CC39408
:101D900064F55B8003755B00E55B75F00284FF7E94
:101DA000008F5BEFC394335007EF24CDF55B8003C6
:101DB000755BFF801CE54475F00284FF7E00900196
:101DC0004E12001EE075F00284FF7E00EF24CDF578
:101DD0005BE595C3955B4004C2A28002D2A2A20734
:101DE000B34005E555B407037570CDE595C395700F
:101DF0004004C2A18002D2A1E542C394064003027E
:101E00002456A2EDB35003022456C2EDE54260030E
:101E1000021F5D7E017F00E5BE1240D8E5BD2FFFA9
:101E200050010E900000EEF0A3EFF0900029E0B416
:101E300001177E0F7FFF900000E0FCA3E0FD120081
:101E400003900000EEF0A3EFF0900079E0B4025BA5
:101E5000900000E0FEA3E0FF90000AE0FCA3E0FD9C
:101E6000EDD39FEC9E400F900000E0F8A3E09000BF
:101E70000AC8F0A3C8F0900000E0FEA3E0FF9000C5
:101E80000CE0FCA3E0FDEFD39DEE9C400F90000022
:101E9000E0F8A3E090000CC8F0A3C8F0900000E0C8
:101EA000FEA3E0FF74041240CA8F43900079E070F3
:101EB00060900000E0FEA3E0FF90000AE0FCA3E0D9
:101EC000FDEFD39DEE9C400D120003900000EEF05C
:101ED000A3EFF08007900000E4F0A3F0900000E092
:101EE000FEA3E0FF74101240D8900026E08E048F0D
:101EF00005FF1240BA900000ECF0A3EDF07400D39F
:101F00009D74019C4008900001E0F54380037543F7
:101F1000FFE54375F00AA4FFAEF074198E048F0537
:101F2000FF1240BA8D44ED2531FFAE3050010E74E2
:101F3000011240CA8F44854431753000EFD394625A
:101F40004003754462900072E06401600690006690
:101F5000E060028005754201800375BB17E542B45D
:101F60000102800302204D7E017F00E5BE1240D8B1
:101F7000E5BD2FFF50010E900000EEF0A3EFF090B2
:101F80000072E0B4017EE53345326025AC32AD33FA
:101F90001DBDFF011C8F028E038C068D07903D78BE
:101FA00012002EE493FE740193FFEFC39AEE9B4060
:101FB0000280057832124102AE32AF3374B3BE00F4
:101FC00025D39F4021900000E0FCA3E0FD0FBF005F
:101FD000010E903D7812002EE493FE740193FFED04
:101FE000C39FEC9E40028005783212003FAE32AFB4
:101FF00033E5691240D874648E048F05FF1240BA2D
:102000008D468033900066E0602D900000E0FEA3D6
:10201000E0FFEFD39400EE9408400F900066E0B428
:102020000104C2098002D209800D900066E0B4016B
:1020300004D2098002C209900072E0640260069036
:102040000066E0600575BB168003754202E542B488
:102050000202800302213B7E017F00E5BE1240D8D0
:10206000E5BD2FFF50010E900000EEF0A3EFF090C1
:102070000072E0B4027EE53345326025AC32AD3308
:102080001DBDFF011C8F028E038C068D07903C0E38
:1020900012002EE493FE740193FFEFC39AEE9B406F
:1020A0000280057832124102AE32AF3374B3BE0003
:1020B00025D39F4021900000E0FCA3E0FD0FBF006E
:1020C000010E903C0E12002EE493FE740193FFED7E
:1020D000C39FEC9E40028005783212003FAE32AFC3
:1020E00033E5691240D874648E048F05FF1240BA3C
:1020F0008D468033900066E0602D900000E0FEA3E6
:10210000E0FFEFD39400EE9408400F900066E0B437
:102110000104C2098002D209800D900066E0B4017A
:1021200004D2098002C209900072E0700375460073
:10213000900066E07002C20975BB1FE542B403451A
:102140007E017F00E5BE1240D8E5BD2FFF50010E95
:10215000900000EEF0A3EFF074091240D874E68E00
:10216000048F05FF1240BA8C408D41E5492DFD508A
:10217000010C74018C068D071240CA8E408F418578
:10218000414975BB19E542B40402800302233E7E37
:10219000017F00E5BE1240D8E5BD2FFF50010E9033
:1021A0000000EEF0A3EFF074041240CA8F4AE5631A
:1021B000B401028003022270756A00756A00E56A44
:1021C000D39407400302225DE56A9000411240F07B
:1021D000E0D3954A501AE56A9000411240F0E0F4CD
:1021E00004254AFEE56A9000371240F0EEF08017B1
:1021F000E56A9000411240F0E0C3954AFEE56A901E
:1022000000371240F0EEF0E56AC3940440099000F4
:1022100084E0C3956A503BE56A6029E56A9000371F
:102220001240F0FEE0FFEE90003FE0D39F4013E548
:102230006A9000371240F0E090003FF0E56A9000AD
:1022400040F0800E900037E090003FF07400900066
:1022500040F0786A740126F640030221BE900040E7
:10226000E0F4042408F555E555D394054002C292E4
:10227000E563D39401402FE54AD3946E4004D20D18
:102280008002C20D755505E563B40205A20DB34089
:10229000028003755507E563B40306A20DB3B3408E
:1022A000028003755507E55665556008E55004F54D
:1022B00051855556E555902686F82828738050D2CA
:1022C000A0804CE543C394585004D2A08002C2A021
:1022D000803DE550C394045007E543C39458400241
:1022E0008004D2A08002C2A080258023E550C39440
:1022F000045007E543C3945840028004D2A08002F2
:0F230000C2A0E550B40402D2A080048002800085
:102686000222BD0222BF0222C30222D20222EA0293
:0B26960022EC02230B02230D02230F95
:10230F00E555B40708E5B54480F5B58006E5B55445
:10231F007FF5B5E55564066005E555B40808E5B5E4
:10232F004410F5B58006E5B554EFF5B575BB13E56B
:10233F0042B4050280030224527E017F00E5BE12E3
:10234F0040D8E5BD2FFF50010E900000EEF0A3EF37
:10235F00F074041240CA8F45E562B4020280030292
:10236F00244F756A00756A00E56AD394034003022F
:10237F002406E56A9000331240F0E0D39545501AD9
:10238F00E56A9000331240F0E0F4042545FEE56A5B
:10239F0090002D1240F0EEF08017E56A9000331296
:1023AF0040F0E0C39545FEE56A90002D1240F0EE37
:1023BF00F0E56A6029E56A90002D1240F0FEE0FF1B
:1023CF00EE900031E0D39F4013E56A90002D12404C
:1023DF00F0E0900031F0E56A900032F0800E90004E
:1023EF002DE0900031F07400900032F0786A7401A3
:1023FF0026F64003022377900082E07043E52945DB
:10240F00286036E557C39403500A900032E004C3A6
:10241F00940340028007900032E004F557E557D34C
:10242F009402400A900032E004D3940250028007D5
:10243F00900032E004F5578007900032E004F55722
:10244F0075BB180542D2ECE55DD394045003022509
:10245F003E75CF01C2A2AE34AF357488D39F7413CB
:10246F009E4005A2A5B34014AE34AF357488D39FF8
:10247F0074139E4005A2A4B3400280487834120022
:10248F003FAE34AF35EFB4883BEEB41337A2A5B3EC
:10249F00500990004FE0D3955050028004055080B2
:1024AF0011A2A5B3500890004FE065506002800262
:1024BF00D207A2A4B35007E550D394015002800471
:1024CF001550C207A2A5B3B35006A2A4B3B34002DE
:1024DF008006753500753400E55065516035E5505F
:1024EF0075F040A4FFAEF090032212001EE030E022
:1024FF0003D38001C39296E55075F040A4FFAEF070
:10250F0090032312001EE030E003D38001C39295A5
:10251F00855051A20740057570CD80037570FFE59A
:10252F0095C395704004C2A18002D2A1022460AE6F
:10253F0024AF25EFD39420EE944E50030226391288
:10254F000481C28E758D00758B00754B00D28EC2C3
:10255F0007756F00756E007570CD7550047523008B
:10256F00752200755300755900C287900059E060BD
:10257F0004D2908002C29090004AE0B40104D29439
:10258F008002C294900049E0B40104D2938002C249
:10259F0093A209B34004D2918002C29190006BE0E4
:1025AF00601812372DA200B34008E5B54408F5B501
:1025BF008006E5B554F7F5B58002C20090006EE0D5
:1025CF006018123882A202B34008E5B54402F5B58F
:1025DF008006E5B554FDF5B58006E5B554FDF5B5B6
:1025EF0090000E74FDF0A374E8F0E542B406037595
:1025FF004200900025E4F0752500752400758D00CC
:10260F00758B00754B00900024E0C3940350089025
:10261F000024E004F080067403900024F09000245E
:10262F00E0B40306E5B554FEF5B5AE26AF27EFD3FC
:10263F009410EE9427401CC2CA75CD0075CC00755E
:10264F002700752600D2CA754D0075290075280020
:06265F00755400020CB0EE
:103A340000000100013201640196019602000212A5
:103A440002240200020003000340038003C00400B8
:103A54000440048004C005000600060006000600B9
:103A6400060006000600060000FF0131016301950F
:103A740001FF01FF0211022302FF02FF02FF033FC5
:103A8400037F03BF03FF043F047F04BF04FF05FF5C
:103A940006FF06FF06FF06FF06FF06FF06FF06FFFA
:103AA4000FAA0FA50F9F0F9A0F940F8D0F870F80EA
:103AB4000F780F710F680F600F570F4E0F450F3BB4
:103AC4000F300F250F1A0F0E0F020EF50EE80EDB46
:103AD4000ECC0EBE0EAE0E9F0E8E0E7D0E6C0E5ACA
:103AE4000E470E340E200E0C0DF70DE20DCB0DB566
:103AF4000D9D0D850D6D0D540D3A0D200D050CE930
:103B04000CCE0CB10C940C760C580C3A0C1B0BFB21
:103B14000BDB0BBB0B9A0B790B570B350B130AF111
:103B24000ACE0AAB0A870A640A400A1C09F809D4B7
:103B340009B0098C09670943091F08FB08D608B2B4
:103B4400088E086A0846082307FF07DC07B90796AA
:103B540007730751072F070D06EC06CA06AA068944
:103B640006690649062A060A05EC05CD05B0059244
:103B740005750558053C0520050504EA04CF04B580
:103B8400049C04820469045104390422040B03F4E0
:103B940003DE03C803B2039D038903750361034D68
:103BA400033B03280316030402F202E102D102C01C
:103BB40002B002A002910282027302650257024916
:103BC400023C022F02220216020901FD01F201E663
:103BD40001DB01D001C601BB01B101A7019D019424
:103BE400018B018201790170016801600158015063
:103BF4000148014101390132012B0125011E01183F
:103C04000111010B010500FF00FA0FA60FA00F9987
:103C14000F920F8B0F840F7C0F740F6B0F620F5872
:103C24000F4E0F430F380F2C0F1F0F120F050EF7F7
:103C34000EE80ED80EC80EB70EA50E930E800E6CAD
:103C44000E580E420E2C0E150DFD0DE40DCB0DB1CC
:103C54000D950D790D5D0D3F0D200D010CE10CC08E
:103C64000C9E0C7C0C590C350C100BEA0BC40B9EEF
:103C74000B760B4F0B260AFD0AD40AAA0A800A55B2
:103C84000A2A09FF09D409A8097C0950092508F959
:103C940008CD08A10875084A081E07F307C8079D40
:103CA40007730749072006F706CE06A6067E0657C1
:103CB4000630060A05E405BF059B05770554053261
:103CC400051004EF04CE04AE048F047104530435CC
:103CD400041903FD03E203C703AD0394037B0363E9
:103CE400034B0334031E030802F302DE02CA02B6C6
:103CF40002A30291027F026D025C024C023C022C80
:103D0400021D020E020001F201E401D701CA01BE44
:103D140001B101A6019A018F0185017A0170016642
:103D2400015D0153014A0141013901310129012198
:103D340001190112010B010400FD00F700F000EA73
:103D440000E400DE00D900D300CE00C900C400BFE7
:103D540000BA00B500B100AD00A800A400A0009C0A
:103D6400009900950091008E008A008700840081EC
:043D7400007E007B52
:1026A100751A00751900AE19AF1AAC17AD18EDC344
:1026B1009FEC9E401674FF1240AA75CF01781A74E0
:1026C1000126F6500418E436F650DB22900786E422
:1026D100F0A3F0751000750F00751300751400C29A
:1026E1000ED20F22C2AF75D900758F0375B7A575CC
:1026F100B7F190F800E4F0758F0175B7A575B7F1E2
:10270100E50890F800F075B7A575B7F190F801E408
:10271100F075B7A575B7F190079DE090F802F075D7
:10272100B7A575B7F19007A1E090F803F075B7A5CB
:1027310075B7F190079EE090F804F075B7A575B7ED
:10274100F190079FE090F805F075B7A575B7F19086
:1027510007A0E090F806F075B7A575B7F19007A24C
:10276100E090F807F0758F0075D940D2AF2290073D
:1027710088E0B4AB61C2AF75D90075B62275F52298
:10278100758F0375B7A575B7F1740090F600F075F4
:102791008F01750A00750900AE09AF0A7413BE00F6
:1027A100279F402475B7A575B7F190078912001EC0
:1027B100E0FC90F60012001EECF0780A740126F697
:1027C100500418E436F650D0758F0075F51175B6C2
:1027D1002075D940D2AF22C2AF75D90075F52275E7
:1027E1000A00750900AE09AF0A7413BE00229F40AA
:1027F1001F90F60012001EE493FC90078912001E40
:10280100ECF0780A740126F6500418E436F650D537
:1028110075F51175D940D2AF22900788E0B4AA02AC
:102821008003022957C2AF75D90075B62275F5220A
:10283100758F0375B7A575B7F1740090EE00F0754B
:10284100B7A575B7F1740090F000F075B7A575B72D
:10285100F1740090F200F075B7A575B7F1740090AE
:10286100F400F0758F01750A00750900AE09AF0A11
:1028710074FFC39F74019E402475B7A575B7F1908D
:10288100004E12001EE0FC90EE0012001EECF078EB
:102891000A740126F6500418E436F650CF750A0082
:1028A100750900AE09AF0A74FFC39F74019E4024ED
:1028B10075B7A575B7F190024E12001EE0FC90F0BD
:1028C1000012001EECF0780A740126F6500418E498
:1028D10036F650CF750A00750900AE09AF0A74FFCC
:1028E100C39F74019E402475B7A575B7F190044E3E
:1028F10012001EE0FC90F20012001EECF0780A7447
:102901000126F6500418E436F650CF750A00750911
:1029110000AE09AF0A74FFC39F74019E402475B7CE
:10292100A575B7F190064E12001EE0FC90F400125E
:10293100001EECF0780A740126F6500418E436F60D
:1029410050CF758F0075F51175B62075D940D2AF8E
:10295100743A90074EF022900788E0B4AA028003EF
:10296100022A95C2AF75D90075B62275F522758F09
:102971000375B7A575B7F1740090E600F075B7A5BA
:1029810075B7F1740090E800F075B7A575B7F174EB
:102991000090EA00F075B7A575B7F1740090EC00EE
:1029A100F0758F01750A00750900AE09AF0A74FF51
:1029B100C39F74019E402475B7A575B7F190004E71
:1029C10012001EE0FC90E60012001EECF0780A7482
:1029D1000126F6500418E436F650CF750A00750941
:1029E10000AE09AF0A74FFC39F74019E402475B7FE
:1029F100A575B7F190024E12001EE0FC90E800129E
:102A0100001EECF0780A740126F6500418E436F63C
:102A110050CF750A00750900AE09AF0A74FFC39F54
:102A210074019E402475B7A575B7F190044E12004C
:102A31001EE0FC90EA0012001EECF0780A740126F8
:102A4100F6500418E436F650CF750A00750900AE49
:102A510009AF0A74FFC39F74019E402475B7A57521
:102A6100B7F190064E12001EE0FC90EC0012001E21
:102A7100ECF0780A740126F6500418E436F650CFCB
:102A8100758F0075F51175B62075D940D2AF743ABE
:102A910090074EF022900788E0B4AA028003022B2F
:102AA100D3C2AF75D90075B62275F522758F03753E
:102AB100B7A575B7F1740090DE00F075B7A575B7CD
:102AC100F1740090E000F075B7A575B7F17400904E
:102AD100E200F075B7A575B7F1740090E400F075E8
:102AE1008F01750A00750900AE09AF0A74FFC39F13
:102AF10074019E402475B7A575B7F190004E120080
:102B01001EE0FC90DE0012001EECF0780A74012633
:102B1100F6500418E436F650CF750A00750900AE78
:102B210009AF0A74FFC39F74019E402475B7A57550
:102B3100B7F190024E12001EE0FC90E00012001E60
:102B4100ECF0780A740126F6500418E436F650CFFA
:102B5100750A00750900AE09AF0A74FFC39F7401BD
:102B61009E402475B7A575B7F190044E12001EE082
:102B7100FC90E20012001EECF0780A740126F65077
:102B81000418E436F650CF750A00750900AE09AF96
:102B91000A74FFC39F74019E402475B7A575B7F1F0
:102BA10090064E12001EE0FC90E40012001EECF0B4
:102BB100780A740126F6500418E436F650CF758F62
:102BC1000075F51175B62075D940D2AF743A9007EA
:102BD1004EF022900788E0B4AA028003022D11C2B0
:102BE100AF75D90075B62275F522758F0375B7A536
:102BF10075B7F1740090D600F075B7A575B7F1748B
:102C01000090D800F075B7A575B7F1740090DA009F
:102C1100F075B7A575B7F1740090DC00F0758F0100
:102C2100750A00750900AE09AF0A74FFC39F7401EC
:102C31009E402475B7A575B7F190004E12001EE0B5
:102C4100FC90D60012001EECF0780A740126F650B2
:102C51000418E436F650CF750A00750900AE09AFC5
:102C61000A74FFC39F74019E402475B7A575B7F11F
:102C710090024E12001EE0FC90D80012001EECF0F3
:102C8100780A740126F6500418E436F650CF750A16
:102C910000750900AE09AF0A74FFC39F74019E401D
:102CA1002475B7A575B7F190044E12001EE0FC9093
:102CB100DA0012001EECF0780A740126F6500418AE
:102CC100E436F650CF750A00750900AE09AF0A74F3
:102CD100FFC39F74019E402475B7A575B7F1900697
:102CE1004E12001EE0FC90DC0012001EECF0780A8F
:102CF100740126F6500418E436F650CF758F00752E
:102D0100F51175B62075D940D2AF743A90074EF0DF
:102D110022C2AF75D90075F522750A00750900AE9A
:102D210009AF0A74FFC39F74019E401F90EE001209
:102D3100001EE493FC90004E12001EECF0780A7421
:102D41000126F6500418E436F650D4750A007509C8
:102D510000AE09AF0A74FFC39F74019E401F90F03B
:102D61000012001EE493FC90024E12001EECF0785B
:102D71000A740126F6500418E436F650D4750A0098
:102D8100750900AE09AF0A74FFC39F74019E401F0D
:102D910090F20012001EE493FC90044E12001EEC0F
:102DA100F0780A740126F6500418E436F650D4750A
:102DB1000A00750900AE09AF0A74FFC39F74019E32
:102DC100401F90F40012001EE493FC90064E120086
:102DD1001EECF0780A740126F6500418E436F65019
:102DE100D475F51175D940D2AF22C2AF75D900752E
:102DF100F522750A00750900AE09AF0A74FFC39F79
:102E010074019E401F90E60012001EE493FC9000A6
:102E11004E12001EECF0780A740126F6500418E4F4
:102E210036F650D4750A00750900AE09AF0A74FF71
:102E3100C39F74019E401F90E80012001EE493FCA2
:102E410090024E12001EECF0780A740126F650042E
:102E510018E436F650D4750A00750900AE09AF0AB8
:102E610074FFC39F74019E401F90EA0012001EE48C
:102E710093FC90044E12001EECF0780A740126F6C1
:102E8100500418E436F650D4750A00750900AE09ED
:102E9100AF0A74FFC39F74019E401F90EC001200A3
:102EA1001EE493FC90064E12001EECF0780A7401A9
:102EB10026F6500418E436F650D475F51175D9404C
:102EC100D2AF22C2AF75D90075F522750A00750916
:102ED10000AE09AF0A74FFC39F74019E401F90DECC
:102EE1000012001EE493FC90004E12001EECF078DC
:102EF1000A740126F6500418E436F650D4750A0017
:102F0100750900AE09AF0A74FFC39F74019E401F8B
:102F110090E00012001EE493FC90024E12001EECA1
:102F2100F0780A740126F6500418E436F650D47588
:102F31000A00750900AE09AF0A74FFC39F74019EB0
:102F4100401F90E20012001EE493FC90044E120018
:102F51001EECF0780A740126F6500418E436F65097
:102F6100D4750A00750900AE09AF0A74FFC39F74D6
:102F7100019E401F90E40012001EE493FC90064E57
:102F810012001EECF0780A740126F6500418E4369B
:102F9100F650D475F51175D940D2AF22C2AF75D9AB
:102FA1000075F522750A00750900AE09AF0A74FFB4
:102FB100C39F74019E401F90D60012001EE493FC33
:102FC10090004E12001EECF0780A740126F65004AF
:102FD10018E436F650D4750A00750900AE09AF0A37
:102FE10074FFC39F74019E401F90D80012001EE41D
:102FF10093FC90024E12001EECF0780A740126F642
:10300100500418E436F650D4750A00750900AE096B
:10301100AF0A74FFC39F74019E401F90DA00120033
:103021001EE493FC90044E12001EECF0780A740129
:1030310026F6500418E436F650D4750A00750900D6
:10304100AE09AF0A74FFC39F74019E401F90DC005C
:1030510012001EE493FC90064E12001EECF0780A5A
:10306100740126F6500418E436F650D475F511753E
:10307100D940D2AF22E51464046006E59964FF608B
:10308100028031A20E4004D20E8027E5146008743C
:10309100E62514900023F0E513600874F0251390E1
:1030A1000023F0E514B4010280FE751400751300CD
:1030B100C20E8002C20EE5149039D7F82828737524
:1030C1001400E599B4FF03751301E599B4FE037586
:1030D1001302E599B4FD03751303E599B4FC037577
:1030E1001304E599B4FA03751305E599B4FB067564
:1030F1001401120481E599B4F906751404120481CE
:10310100E599D394E54007E599C394F04002801610
:103111008599157514027E017F00E515C394E612A9
:1031210040D88E0D8F0E900786E4F0A3F0E599D379
:1031310094C44007E599C394E64002802885991517
:1031410075140374E5C39515F50E750D00AE0DAF3D
:103151000E903A3412002EE493F87401939007868E
:10316100C8F0A3C8F0D2990235EB900786E0FEA320
:10317100E0FFEFC39400EE94054009EFD394FFEE16
:1031810094064013900786E0FEA3E0FF90004E12E4
:10319100001EE599F0800385996B90078612000E59
:1031A100900786E0FEA3E0FFEFB40106EEB407024C
:1031B10080030233F890074EE0B43C0280030233EF
:1031C100F875FFA0A20AB35005A20BB34003023267
:1031D100EBC29C90007AE090078CF0900057E09051
:1031E100078DF0900062E090078EF0900063E09010
:1031F100078FF0900074E0900790F090007CE090D1
:103201000791F090007DE0900792F0900080E090AF
:103211000793F0900081E0900794F090013AE090DC
:103221000795F090013BE0900796F090013CE0900B
:103231000797F0900090E0900798F0900091E0904F
:103241000799F0900092E090079AF0900093E09037
:10325100079BF0900094E090079CF0900095E0901F
:10326100079DF0900096E090079EF0900097E09007
:10327100079FF0900099E09007A0F090009AE090ED
:1032810007A1F090009BE09007A2F090009CE090D5
:1032910007A3F07400900082F01200C974AB90078C
:0D32A10088F012276F74AA900788F0E55797
:0639D7000230C002316B5A
:1032AE009039F8F8282873801212281A800D1229E6
:0B32BE00588008122A968003122BD4BF
:0F39F8000232B50232B70232BC0232C10232C60D
:1032C900900788E4F090013AE0700C90013BE070BF
:1032D9000690013CE060028004C20A8002D20A0220
:1032E90033EDC29C900078E0900789F090005EE091
:1032F90090078AF090005FE090078BF090007AE0E9
:1033090090078CF0900057E090078DF0900062E0F4
:1033190090078EF0900063E090078FF0900074E0C2
:10332900900790F090007CE0900791F090007DE08C
:10333900900792F0900080E0900793F0900081E070
:10334900900794F090013AE0900795F090013BE0E6
:10335900900796F090013CE0900797F0900090E07C
:10336900900798F0900091E0900799F0900092E012
:1033790090079AF0900093E090079BF0900094E0FA
:1033890090079CF0900095E090079DF0900096E0E2
:1033990090079EF0900097E090079FF0900099E0C9
:1033A9009007A0F090009AE09007A1F090009BE0B0
:1033B9009007A2F090009CE09007A3F074009000A1
:1033C90082F074AB900788F012276F74AA9007886F
:1033D900F012281A122958122A96122BD4D29C7547
:1033E90099FB80FED29C7514007513007599FB0238
:1033F90035EB900786E0FEA3E0FFEF4E7006859956
:1034090010750F00900786E0FEA3E0FF74016F4E70
:10341900701BAC0FAD10AA0DAB0EED2BFBEC3AFAFD
:103429008A068B0790004E12001EE599F0900786D8
:1034390012000E900786E0FEA3E0FF74026F4E7043
:103449000C1200C98515997514007513000235EB26
:10345900900786E0FEA3E0FF90004E12001EE5995A
:10346900F090078612000E900786E0FEA3E0FFACFD
:103479000DAD0E8F028E038C068D07903A6C1200EB
:103489002EE493F9740193FEEAD39EEB99400985E2
:1034990015997514007513000235EB900786E0FE47
:1034A900A3E0FF90004E12001EE599F090078612E6
:1034B900000E900786E0FEA3E0FFEFB40006EEB42D
:1034C900010280030235EB75FFA090001CE0D39444
:1034D900C7400B90001CE0C394C8F516801A9000F1
:1034E9001CE0D39463400B90001CE0C39464F51670
:1034F900800690001CE0F516E51675F002A4FFAEF3
:10350900F08F6AEF90004E1240F0EFFCE0FDEC9076
:1035190000511240F0EDFCE0FDEC2DB516028003E0
:103529000235DD0FEF90004E1240F0E56AFFE0FC36
:10353900EF9000521240F0ECFFE0FCEFC39CB5168F
:103549000280030235DDE56A9000501240F0E56A19
:10355900FFE0FCEF9000531240F0ECFFE0FCEF2C91
:10356900B51671E56A9000541240F0E0C3951690C3
:10357900079DF0E56A9000551240F0E0C39516905A
:10358900079EF0E56A9000581240F0E0C395169046
:10359900079FF0E56A9000591240F0E0C395169034
:1035A90007A0F0E56A90005A1240F0E0C395169022
:1035B90007A1F0E56A90005B1240F0E0C395169010
:1035C90007A2F01226E57599F975186475170012A6
:1035D90026A180FE7599FF7518647517001226A13A
:0235E90080FE62
:0939DD000233FB0234590234A448
:1035EB0022E5139039E6F828287302372C900786CA
:1035FB00E0FEA3E0FF90001212001EE0F599900789
:10360B008612000E900786E0FEA3E0FF74116F4E4A
:10361B00700375130002372C85619902372C9007C4
:10362B0086E0FEA3E0FF90004E12001EE0F599EF3E
:10363B00B40107EEB4070375130090078612000E52
:07364B0002372C900787E015
:0F39E6000235F50235F802362302362902364E35
:10365200903A07F8282873852399023721852999FA
:103662000237218543990237218546990237218500
:103672005099023721855F99023721855599023782
:1036820021855799023721756D00900069E0700617
:10369200900068E060028016A2A44006E56D440432
:1036A200F56DA2A54006E56D4402F56D801A900005
:1036B2004AE0B40106E56D4410F56D900049E0B4AE
:1036C2000106E56D4420F56DA207B34006E56D44A1
:1036D20001F56DA209B34006E56D4408F56D856DEF
:1036E20099803CA20FB340077599FAC20F8017A2C6
:1036F2000CB3400575990F800B900023E0F599906B
:103702000023E4F0C20C80178541998012854A9902
:0F371200800D85459980087599FC80037513001B
:103A070002365902365F02366502366B023671029C
:103A1700367702367D0236830236890236E502376B
:0D3A27000A02370F02371402371902371E4A
:0B37210090078612000E800312004883
:0339F5000237296D
:10372C002290006BE0B4010385231190006BE0B490
:10373C00020385291190006BE0B4030385431190BB
:10374C00006BE0B4040385461190006BE0B40503F4
:10375C0085501190006BE0B4060385551190006BF9
:10376C00E0B4070385571190006CE0FE90006DE00B
:10377C00C39E500302380390006BE0D39404402C9A
:10378C0090006CE0D39511500990006DE0C3951139
:10379C0050028002D20090006CE0D3951150099039
:1037AC00006DE0C395115002C200804990006BE09F
:1037BC00B4041890006DE0C395115002D200900033
:1037CC006CE0D395114002C200802A90006CE0C3DB
:1037DC009511500990006DE0D3951150028002D2E2
:1037EC000090006CE0D39511500990006DE0C395EA
:1037FC00115002C200807E90006BE0D39404402CE8
:10380C0090006CE0C39511400990006DE0D39511C8
:10381C0040028002C20090006CE0C39511400990F8
:10382C00006DE0D395114002D200804990006BE00E
:10383C00B4041890006CE0C395115002C2009000C3
:10384C006DE0D395114002D200802A90006CE0C349
:10385C009511400990006DE0D395114002D2009073
:10386C00006CE0D39511400990006DE0C3951140B8
:10387C00028002C2002290006EE0B4010385231185
:10388C0090006EE0B4020385291190006EE0B40341
:10389C000385431190006EE0B4040385461190003B
:1038AC006EE0B4050385501190006EE0B4060385FC
:1038BC00551190006EE0B4070385571190006FE02E
:1038CC00FE900070E0C39E500302395890006EE0E9
:1038DC00D39404402C90006FE0D3951150099000C4
:1038EC0070E0C3951150028002D20290006FE0D3B9
:1038FC0095115009900070E0C395115002C20280DE
:10390C004990006EE0B40418900070E0C39511501B
:10391C0002D20290006FE0D395114002C202802ABD
:10392C0090006FE0C395115009900070E0D3951191
:10393C0050028002D20290006FE0D3951150099092
:10394C000070E0C395115002C202807E90006EE0C0
:10395C00D39404402C90006FE0C395114009900063
:10396C0070E0D3951140028002C20290006FE0C358
:10397C0095114009900070E0D395114002D202805D
:10398C004990006EE0B4041890006FE0C39511509C
:10399C0002C202900070E0D395114002D202802A3C
:1039AC0090006FE0C395114009900070E0D3951121
:1039BC004002D20290006FE0D39511400990007044
:0B39CC00E0C3951140028002C20222FD
:0940F0002582F5825002058322AD
:10002E00EF2F500205832582F582E5833E2EF58360
:01003E00229F
:08000300C3EF9DFFEE9CFE22FD
:08003F000806B60002180622B3
:0D000E00A3E004F070061240E6E004F022CA
:084102000816B6FF0218162290
:0E40CA00048007C3CE13CECF13CFD5E0F6226D
:103F7800BC000FBE0008ED8FF084FFADF022E4FE18
:103F8800FF22BE000DEF60FE54F0606F20E70302D1
:103F9800402EEAC0E0EBC0E078017A0075F001EE4F
:103FA80020E710EF25E0FFEE33FE0AC5F023C5F049
:103FB80030E7F0EA5407F9096A7A007B00600108E3
:103FC800C3EC9E40167004ED9F4010ED9FFDEC9EE3
:103FD800FCE5F0CA4ACA03F5F08005E5F003F5F000
:103FE800C3EE13FEEF13FFD9D77908CACBCAD8D0CE
:103FF800EAFEEBFFD0E0FBD0E0FA22EC8FF084FC85
:10400800ED54F045F0C48FF084FEEDC454F045F053
:10401800C48FF084FDEEC4FE54F02DFFEE540F3C27
:10402800FEADF07C0022790078008FF0EC7E08204D
:10403800E70DC3CD33CD33C933C9C833C8DEF084E7
:1040480049F9E5F08FF0BE00E6FD7C00E9FFE8FEE7
:014058002245
:0E40D800F88FF0A4FFE5F0CE88F0A42EFE22B3
:1040AA00600D782B0240B4007830D8FED5E0F822B3
:1040BA00EEC0E07E00123F78EFFDEEFCD0E0FE227B
:03000B0002405957
:03001B000240742C
:03002B0002408F01
:030000000240F9C2
:0940F90075817175D0000207EA1F
:0B001E00E5822FF582E5833EF583228A
:0A40E6000582D5820215831582229F
:10405900C0E0C0F0C083C082C0D075D0001207DFB5
:10406900D0D0D082D083D0F0D0E032C0E0C0F0C050
:1040790083C082C0D075D0001207E2D0D0D082D0E0
:1040890083D0F0D0E032C0E0C0F0C083C082C0D09D
:1040990075D0001207E5D0D0D082D083D0F0D0E01F
:0140A90032E4
:00000001FF
